:100000000C944A050C9491050C9491050C9491055F
:100010000C9491050C9491050C9491050C94910508
:100020000C9491050C9491050C9491050C94FB0B88
:100030000C94AA0C0C94011B0C9491050C94910542
:100040000C9491050C9491050C9491050C94751BDE
:100050000C9491050C9491050C9491050C949105C8
:100060000C9491050C9491050C9491050C949105B8
:100070000C94910589068C068F06920695069806C3
:100080009B06170D390D270E390D270E7E0DA10D7C
:10009000270EF60D090EA811A811D611D61133128C
:1000A00071128A148A148A128A148B138B135E14A9
:1000B0008A148A1475147E10360E0F12272D7F377E
:1000C000383334132F2E7C7D29283130742A7879E7
:1000D00039042B14351E7B641D161A081F207A1B49
:1000E0000709151721222C06190A1C182324650557
:1000F000110B0D0C25260A002530325800626F7551
:100100006E6365213A20004B6579626F61726420ED
:1001100073746172742E0A0055534220636F6E66C9
:100120006967757265642E0A000D0A696E69740A42
:10013000000E0341006C00700073003600340000B4
:1001400000080354004D004B00000004030904099B
:10015000027400040100A03209040000010301013F
:100160000009211101000122400007058103080058
:100170000A09040100010301020009211101000123
:10018000224D000705820308000A0904020001034A
:100190000000000921110100012236000705830338
:1001A00008000A09040300020300000009211101EC
:1001B0000001222200070584032000010705040333
:1001C0002000011201100100000008EDFE6464012E
:1001D00000010200010631FF0974A1010975150033
:1001E00026FF009520750881020976150026FF007C
:1001F000952075089102C005010980A101850216AC
:10020000810026B7001A81002AB700751095018178
:1002100000C0050C0901A1018503160100269C02FE
:100220001A01002A9C02751095018100C005010980
:1002300002A1010901A100050919012905150025DF
:10024000019505750181029501750381010501097B
:100250003009311581257F95027508810609381509
:1002600081257F950175088106050C0A38021581E4
:10027000257F950175088106C0C005010906A10109
:10028000050719E029E71500250195087501810288
:100290009501750881010508190129059505750164
:1002A00091029501750391010507190029FF1500B9
:1002B00026FF00950675088100C0636F6E73756D2B
:1002C00065723A20253034580A0073797374656D6D
:1002D0003A20253034580A000A00253032582000D0
:1002E0006B6579626F6172643A20004C45443A2034
:1002F000253032580A00253032583A2025303862ED
:1003000025730A00722F632030313233343536378B
:100310000A00646F6E652E0A00626F6F746D61670C
:100320006963207363616E3A202E2E2E2000290A05
:10033000002575002F002575005D2800256400202C
:1003400000256400200025640020002564007C0056
:1003500025303258006D6F7573656B6579205B626F
:10036000746E7C782079207620685D287265702F05
:1003700061636C293A205B006D6B5F776865656C23
:100380005F74696D655F746F5F6D6178203D2025D6
:10039000640A006D6B5F776865656C5F6D61785F9F
:1003A0007370656564203D2025640A006D6B5F7481
:1003B000696D655F746F5F6D6178203D2025640A0B
:1003C000006D6B5F6D61785F7370656564203D20C3
:1003D00025640A006D6B5F696E74657276616C20CE
:1003E0003D2025640A006D6B5F64656C6179203D7A
:1003F0002025640A006D6B5F776865656C5F7469C2
:100400006D655F746F5F6D6178203D2025640A0023
:100410006D6B5F776865656C5F6D61785F73706544
:100420006564203D2025640A006D6B5F74696D650D
:100430005F746F5F6D6178203D2025640A006D6BED
:100440005F6D61785F7370656564203D2025640A87
:10045000006D6B5F696E74657276616C203D20255E
:10046000640A006D6B5F64656C6179203D202564D2
:100470000A000A00257500363A20776865656C5FCA
:1004800074696D655F746F5F6D61783A20000A0072
:10049000257500353A20776865656C5F6D61785F1A
:1004A00073706565643A20000A00257500343A20AF
:1004B00074696D655F746F5F6D61783A20000A0042
:1004C000257500333A206D61785F73706565643A15
:1004D00020000A00257500323A20696E7465727634
:1004E000616C286D73293A20000A00257500313AA5
:1004F0002064656C6179282A31306D73293A2000B7
:100500000A092D2056616C756573202D0A004D3E39
:10051000004D25643E20003F0073657420646566CD
:1005200061756C740A00433E20007768657265202F
:1005300064656C74613A20637572736F723D2564F3
:100540002C20776865656C3D25640A5365652068D5
:100550007474703A2F2F656E2E77696B69706564BD
:1005600069612E6F72672F77696B692F4D6F757395
:10057000655F6B6579730A000A092D204D6F7573ED
:10058000656B6579202D0A4553432F713A097175C2
:1005900069740A313A0964656C6179282A31306DD1
:1005A00073290A323A09696E74657276616C286D36
:1005B00073290A333A096D61785F73706565640A5F
:1005C000343A0974696D655F746F5F6D61780A35DF
:1005D0003A09776865656C5F6D61785F7370656512
:1005E000640A363A09776865656C5F74696D655FA2
:1005F000746F5F6D61780A0A703A097072696E747F
:100600002076616C7565730A643A097365742064B9
:10061000656661756C74730A75703A092B310A64EA
:100620006F776E3A092D310A706775703A092B3170
:10063000300A7067646F776E3A092D31300A0A7399
:1006400070656564203D2064656C7461202A206DAE
:1006500061785F7370656564202A20287265706513
:100660006174202F2074696D655F746F5F6D6178B0
:10067000290A003F004D3E2000433E20004C2564E7
:100680000A000A092D20436F6E736F6C65202D0AD6
:100690004553432F713A09717569740A6D3A096DB2
:1006A0006F7573656B65790A000A092D204D6167C6
:1006B0006963202D0A643A0964656275670A783AAD
:1006C000096465627567206D61747269780A6B3AB6
:1006D000096465627567206B6579626F6172640A8F
:1006E0006D3A096465627567206D6F7573650A768A
:1006F0003A0976657273696F6E0A733A09737461A9
:100700007475730A633A09636F6E736F6C65206D5D
:100710006F64650A302D343A096C61796572302D49
:1007200034284631302D4634290A506175733A0910
:10073000626F6F746C6F616465720A653A09656512
:1007400070726F6D0A000A002575002E6E6B726F55
:100750003A20000A002575002E737761705F626190
:10076000636B736C6173685F6261636B7370616309
:10077000653A20000A002575002E737761705F6767
:10078000726176655F6573633A20000A0025750023
:100790002E6E6F5F6775693A20000A002575002E7E
:1007A000737761705F72616C745F726775693A200C
:1007B000000A002575002E737761705F6C616C74A0
:1007C0005F6C6775693A20000A002575002E636129
:1007D00070736C6F636B5F746F5F636F6E74726F57
:1007E0006C3A20000A002575002E737761705F63F4
:1007F0006F6E74726F6C5F636170736C6F636B3A72
:1008000020000A0025303258006B65796D61705FF9
:10081000636F6E6669672E7261773A20000A002561
:1008200075002E6D6F7573653A20000A00257500FE
:100830002E6B6579626F6172643A20000A0025753B
:10084000002E6D61747269783A20000A00257500E7
:100850002E656E61626C653A20000A0025303258C0
:100860000064656275675F636F6E6669672E7261AB
:10087000773A20000A0025750064656661756C741E
:100880005F6C617965723A20003F0074696D657232
:100890005F72656164333228293A202530346C5800
:1008A0000A006B6579626F6172645F69646C653AB6
:1008B0002025580A006B6579626F6172645F7072FF
:1008C0006F746F636F6C3A2025580A00686F7374F9
:1008D0005F6B6579626F6172645F6C656473282910
:1008E0003A2025580A000A092D2053746174757343
:1008F000202D0A004743433A20342E392E3220411E
:1009000056522D4C4942433A20312E382E307376C0
:100910006E204156525F415243483A20617672330D
:10092000350A004F5054494F4E533A204C554641DA
:1009300020424F4F544D41474943204D4F55534559
:100940004B45592045585452414B455920434F4E31
:10095000534F4C4520434F4D4D414E44204B45593C
:100960004D41505F53454354494F4E203430393642
:100970000A004255494C443A2063306630393039D8
:100980002D6469727479202831343A32303A35391D
:10099000204A616E2031312032303137290A005629
:1009A00049443A2030784645454428544D4B292047
:1009B0005049443A2030783634363428416C7073CC
:1009C000363429205645523A203078303030310ABA
:1009D00000444553433A20544D4B206B6579626F78
:1009E000617264206669726D7761726520666F72EC
:1009F00020416C707336340A000A092D2056657246
:100A000073696F6E202D0A000A6D6F7573653A2049
:100A10006F66660A000A6D6F7573653A206F6E0A1D
:100A2000000A6B6579626F6172643A206F66660ACC
:100A3000000A6B6579626F6172643A206F6E0A001A
:100A40000A6D61747269783A206F66660A000A6DF1
:100A500061747269783A206F6E0A000A6465627583
:100A6000673A206F6E0A000A64656275673A206F04
:100A700066660A000A0A626F6F746C6F6164657261
:100A80002E2E2E2000433E20006565636F6E666942
:100A9000673A0A0011241FBECFEFD4E0DEBFCDBFFE
:100AA00004B603FE27C08091CD019091CE01A091A4
:100AB000CF01B091D0018730904BA740B04BD1F41B
:100AC0001092CD011092CE011092CF011092D00160
:100AD00014BE84B7877F84BF0FB6F894A895809121
:100AE0006000886180936000109260000FBEE0E0BB
:100AF000F8E3099511E0A0E0B1E0ECE8FEE402C003
:100B000005900D92A433B107D9F721E0A4E3B1E039
:100B100001C01D92AD3CB207E1F70E9447090C9459
:100B200044270C940000FF93EF93E0913401F0917F
:100B30003501309709F00995EF91FF910895FC0177
:100B40008591803011F0EFDFFBCF0895FF27E0E2C1
:100B500030E247FF0CC0419597FF09C0EDE2609578
:100B6000709580959095611D711D811D911D27FFC8
:100B700002C0219530E350E2AA27660F771F881F35
:100B8000991FAA1FA41710F0A41B63955A95A9F7E3
:100B9000AA3008F0A95FA05DAF93F39561157105C8
:100BA0008105910541F7ED3211F4EF93F395F217BA
:100BB00018F43F93F395FBCF8F91B5DFFA95E1F7EA
:100BC0000895E991F9918591803021F0853219F0ED
:100BD000AADFF9CF089520E0E89455915532C1F38A
:100BE000503311F4689455915A3348F4505390F3AC
:100BF000220F022E220F220F200D250FF4CF0EF40C
:100C0000219589919991533619F3533729F1533529
:100C100059F1BC0188279927E8945C3621F4899121
:100C2000999168945591543639F446EF7EF077FFE8
:100C30000DC08FEF9FEF0AC055374AE039F05835A5
:100C400040E121F0523642E009F00895FF93EF931E
:100C50007DDFEF91FF91B7CFFF93EF93FC0181917F
:100C60008030B9F360DFFBCFFF93EF9368DFF1CF04
:100C7000DF93CF93CDB7DEB72596A3DFCF91DF917A
:100C800008958AB180788AB98BB180788BB93A9807
:100C9000429808950E94410684B114B885B18FEF3F
:100CA00085B9A6E3B1E0EEE3F1E088E08E0F1192A2
:100CB0001D928E13FCCF8091AE0182608093AE01B5
:100CC0003D9A459A2FEF89E698E121508040904067
:100CD000E1F700C000003D9845980895EF92FF921B
:100CE0000F931F93CF93DF93C6E3D1E0F12C85E000
:100CF000E82E08EF10E08F2D90E0FC013197E730EF
:100D0000F10520F4E65CFF4F0C94F926509A5898B0
:100D100014C0519A599811C0529A5A980EC0539AB9
:100D20005B980BC0549A5C9808C0559A5D9805C0B2
:100D3000569A5E9802C03A9A429880EA8A95F1F7EC
:100D400083B180959881981739F18883809100014B
:100D5000882301F18091AE0180FF04C08DEF90E007
:100D60000E949F058091AE0180FF0CC08091000120
:100D70001F928F931F930F930E9438060F900F902E
:100D80000F900F908091AE0180FF04C086EF90E03D
:100D90000E949F05E09200010E944106F394219673
:100DA00098E0F912A8CF809100018823B1F081501A
:100DB00080930001882339F08FE99FE00197F1F7D4
:100DC00000C000000AC0AEE3B1E0E6E3F1E0CF010D
:100DD000885F91919D938E13FCCF81E0DF91CF913D
:100DE0001F910F91FF90EF900895E82FF0E0E25CE3
:100DF000FE4F8081089581FF03C03D9A459A089572
:100E00003D98459808958091520108959FB7F894B0
:100E1000109249019FBF9091C301943009F057C0CF
:100E20009091E9009F703091EC00232F217030FDEC
:100E300020E8922B24E02093E9002091EB0020FF92
:100E400043C02091EE0027FF3FC02091460122239E
:100E500021F02091E80025FF37C01092460126E0DE
:100E60003091E80035FD15C03091C301343061F593
:100E70003091EB0035FD28C0215021F481E08093B2
:100E8000460122C0EFE9FFE03197F1F700C0000012
:100E9000E7CF8093F1008091E80085FD0AC0809142
:100EA000E80080FFFCCF8091E8008E778093E80017
:100EB00006C08FB7F89421E0209349018FBF9F703F
:100EC0009093E90080E008959F709093E9008FEF80
:100ED0000895CF93DF9300D01F92CDB7DEB79C016A
:100EE0008091C301843019F593E099833B832A8371
:100EF0009093E9008FEF9091E800815095FD06C036
:100F000095ED9A95F1F700008111F5CF8091E800F9
:100F100085FF0DC040E050E063E070E0CE01019637
:100F20000E94090A8091E8008E778093E8000F9074
:100F30000F900F90DF91CF910895CF93DF9300D062
:100F40001F92CDB7DEB72091C301243021F522E0F6
:100F500029839B838A8383E08093E9008FEF9091BC
:100F6000E800815095FD06C095ED9A95F1F70000D7
:100F70008111F5CF8091E80085FF0DC040E050E081
:100F800063E070E0CE0101960E94090A8091E800BA
:100F90008E778093E8000F900F900F90DF91CF91A4
:100FA00008952091C3012430F1F422E02093E90058
:100FB0002FEF3091E800215035FD06C035ED3A9510
:100FC000F1F700002111F5CF2091E80025FF0BC0BB
:100FD00040E050E065E070E00E94090A8091E8007E
:100FE0008E778093E8000895CF93DF932091C3011B
:100FF000243039F521E02093E9002FEF3091E8000B
:10100000215035FD06C035ED3A95F1F7000021116C
:10101000F5CF2091E80025FF14C0EC0140E050E03E
:1010200068E070E00E94090A8091E8008E77809362
:10103000E80088E0FE01AAE4B1E001900D928A95F3
:10104000E1F7DF91CF9108950895209147012F5F37
:10105000822F62E30E94D926992319F02093470139
:1010600008951092470180914901882371F1809180
:10107000C301843041F58091E9008F702091EC002C
:10108000922F917020FD90E8892B94E09093E900D5
:101090009091EB0090FF14C09091EE0097FF10C06C
:1010A0009091E80095FF03C01092F100F9CF909164
:1010B000E80090FF05C09091E8009E779093E800CB
:1010C0008F708093E90010924901089542E061EC2D
:1010D00081E00E94120B42E061EC82E00E94120B60
:1010E00042E061EC83E00E94120B42E261EC84E09A
:1010F0000C94120B8091C501833009F453C030F475
:10110000813071F0823009F48CC008958A3009F47E
:1011100078C08B3009F45EC0893009F09AC020C0D5
:101120008091C401813A09F094C08091E800877FE2
:101130008093E8008091C8019091C901892B21F426
:1011400068E08AE491E003C060E080E090E070E055
:101150000E94540A8091E8008B778093E8000895FC
:101160008091C401813209F074C08091C8019091CE
:10117000C901892B09F06DC08091E800877F8093B9
:10118000E8008091E80082FD05C08091C3018111D3
:10119000F8CF5FC08091F100809352018091E80008
:1011A0008B7753C08091C401813A09F052C080917D
:1011B000C8019091C901892B09F04BC08091E800CA
:1011C000877F8093E8008091E80080FFFCCF8091CA
:1011D0000B0136C08091C4018132D9F58091C801DC
:1011E0009091C901892BA9F58091E800877F8093B0
:1011F000E8000E94470B8091C60180930B010C947C
:10120000AC148091C401813221F58091E800877F80
:101210008093E8000E94470B8091C701809353019F
:1012200008958091C401813AA1F48091E800877FFC
:101230008093E8008091E80080FFFCCF809153010B
:101240008093F1008091E8008E778093E8000C9401
:10125000470B0895089508958091520180934801A5
:101260001092520180E00E94FB060E94C70F0C946E
:10127000AC140C942C090E94C01A8091C1018823DF
:1012800029F00E94E91A81110C94F309089584B79A
:10129000877F84BF0FB6F894A8958091600088611D
:1012A00080936000109260000FBE90E080E80FB65F
:1012B000F89480936100909361000FBE86E097E000
:1012C0000E94941A89E291E00E949F050E942A09D7
:1012D0000E94000F0E94980B0E94EB0B8091E2008D
:1012E00084608093E20078948091C3018430E1F7B8
:1012F00088E191E00E949F050E94020F81E091E049
:101300000E943F0E87E091E00E949F050E942B09FA
:101310008091C301853019F40E943B09F9CF0E94E6
:10132000080FF6CF0E94FD1A809148018093520168
:1013300008950C949209292F332723303105C9F0E1
:1013400064F42130310581F02230310509F043C0C9
:1013500084E790E02FE431E042C021323105F1F022
:101360002232310541F137C082E190E023EC31E0D7
:1013700036C099278130910541F08230910541F0C6
:10138000892B49F5EBE4F1E005C0E1E4F1E002C0AE
:10139000E1E3F1E0849190E09F0121C06430D8F452
:1013A000E62FF0E0EE0FFF1FE05EFE4F208131815F
:1013B00089E090E014C0643070F470E0FB01EE0F3F
:1013C000FF1FE85EFE4F20813181FB01EC5EFE4F86
:1013D000808190E004C080E090E020E030E0FA01FD
:1013E00031832083089584E089BD86E089BD09B4F6
:1013F00000FEFDCF8091D8008F7D8093D800809132
:10140000E00082608093E0008091E00081FDFCCFED
:101410000895CF92DF92EF92FF920F931F93CF9395
:10142000DF93EC018B016A010E94660B811133C0CE
:10143000C114D10439F0F60180819181081B190B88
:10144000C80FD91FE12CF12C0115110519F180915C
:10145000E80085FD16C08091E8008E778093E80053
:10146000C114D10449F0F60180819181E80EF91E82
:10147000F182E08285E00FC00E94660B882321F391
:101480000AC089918093F10001501109FFEFEF1A12
:10149000FF0ADACF80E0DF91CF911F910F91FF908B
:1014A000EF90DF90CF9008952091CA013091CB0149
:1014B0002617370748F06115710539F42091E800C7
:1014C0002E772093E80001C0B90140E06115710555
:1014D00091F12091C301222309F440C0253009F481
:1014E0003FC02091E80023FD3DC02091E80022FD8F
:1014F0002FC02091E80020FFE9CF2091F20030E0DA
:10150000FC01CF016115710559F02830310540F417
:1015100081918093F100615071092F5F3F4FF1CFAE
:1015200041E02830310509F040E02091E8002E77B5
:101530002093E800CBCF4111CCCF0AC08091C301EA
:10154000882361F0853061F08091E80083FD0AC056
:101550008091E80082FFF2CF80E0089582E0089554
:1015600083E0089581E008952091CA013091CB0174
:101570002617370748F06115710539F42091E80006
:101580002E772093E80001C0B901FC0120E061152D
:10159000710579F18091C301882309F43DC085303C
:1015A00009F43CC08091E80083FD3AC08091E800D6
:1015B00082FD2CC08091E80080FFE9CF8091F2008D
:1015C00090E06115710559F08830910540F424913F
:1015D0002093F1003196615071090196F2CF21E01C
:1015E000089709F020E08091E8008E778093E8006A
:1015F000CECF2111CFCF0AC08091C301882361F0E3
:10160000853061F08091E80083FD0AC08091E80098
:1016100082FFF2CF80E0089582E0089583E008958C
:1016200081E00895982F953058F59093E900981728
:1016300039F07091EC002091ED005091F00003C062
:10164000242F762F50E021FF19C03091EB003E7F10
:101650003093EB003091ED003D7F3093ED00309101
:10166000EB0031603093EB007093EC002093ED00C1
:101670005093F0002091EE0027FF07C09F5FD3CF6B
:101680008F708093E90081E0089580E00895809153
:10169000C40187FF11C08091E80082FD05C08091E0
:1016A000C3018111F8CF11C08091E8008B770BC086
:1016B0008091C301882349F08091E80080FFF8CF32
:1016C0008091E8008E778093E80008952091E400EF
:1016D0003091E50095E64091EC00842F817040FF49
:1016E00022C08091E80080FD1CC08091C301882346
:1016F00091F0853091F08091EB0085FD10C0409114
:10170000E4005091E5004217530729F39A019150E4
:1017100011F784E0089582E0089583E0089581E060
:10172000089580E008954091E80042FFDECF0895DB
:101730000E94F50B0E94F80BE0EEF0E080818160E2
:101740008083E8EDF0E080818F77808319BCE3E649
:10175000F0E08081816080831092C20108950E9430
:10176000F50B0E94F80B8091D8008F778093D800FA
:101770008091D80080688093D8008091D8008F7DB8
:101780008093D80084E089BD86E089BD09B400FE5D
:10179000FDCF1092C3011092BF011092C1011092AF
:1017A000C00142E060E080E00E94120B8091E10005
:1017B0008E7F8093E1008091E20081608093E2005F
:1017C0008091E20088608093E2008091E0008E7F4B
:1017D0008093E0000895E3E6F0E080818E7F8083CF
:1017E00081E08093C2010C94AF0B1092E200089547
:1017F0001092E10008951F920F920FB60F921124DC
:101800002F933F934F935F936F937F938F939F9308
:10181000AF93BF93EF93FF938091E10082FF0BC0E2
:101820008091E20082FF07C08091E1008B7F80936E
:10183000E1000E9425088091E10080FF19C080919D
:10184000E20080FF15C08091E2008E7F8093E2006D
:101850008091E20080618093E2008091D8008062F4
:101860008093D80019BC85E08093C3010E94390998
:101870008091E10084FF30C08091E20084FF2CC0A1
:1018800084E089BD86E089BD09B400FEFDCF80916A
:10189000D8008F7D8093D8008091E1008F7E809367
:1018A000E1008091E2008F7E8093E2008091E2006F
:1018B00081608093E2008091BF01882311F084E071
:1018C00007C08091E30087FD02C081E001C083E092
:1018D0008093C3010E9499098091E10083FF29C090
:1018E0008091E20083FF25C08091E100877F809393
:1018F000E10082E08093C3011092BF018091E1007A
:101900008E7F8093E1008091E2008E7F8093E200E1
:101910008091E20080618093E20042E060E080E03C
:101920000E94120B8091F00088608093F0000E946A
:101930002408FF91EF91BF91AF919F918F917F917B
:101940006F915F914F913F912F910F900FBE0F902C
:101950001F9018951F920F920FB60F9211242F937C
:101960003F934F935F936F937F938F939F93AF9327
:10197000BF93CF93DF93EF93FF93C091E900CF70B4
:101980008091EC00D82FD17080FDD0E81092E90052
:101990008091F000877F8093F00078940E94EE0C95
:1019A0001092E9008091F00088608093F000CD2BC8
:1019B000CF70C093E900FF91EF91DF91CF91BF917C
:1019C000AF919F918F917F916F915F914F913F91D7
:1019D0002F910F900FBE0F901F9018951F93CF93CC
:1019E000DF93CDB7DEB7AA970FB6F894DEBF0FBE70
:1019F000CDBFE4ECF1E088E08E0F9091F10091937F
:101A00008E13FBCF0E947A088091E80083FF1FC1EC
:101A10008091C4019091C501492F50E04A30510591
:101A200008F015C1FA01EF5BFF4F0C94F9268038DE
:101A300081F0823809F00BC18091C8018F708093CA
:101A4000E9008091EB0085FB882780F91092E9007E
:101A500006C08091C0019091C10191118260909166
:101A6000E800977F9093E8008093F1001092F100D6
:101A7000C8C0282F2D7F09F0EAC0882319F08230D2
:101A800061F0E5C08091C601813009F0E0C093307B
:101A900009F080E08093C1012BC08091C6018111C3
:101AA00027C08091C8018F7009F4D1C08093E900EC
:101AB0002091EB0020FF1CC0933021F48091EB00BB
:101AC000806214C09091EB0090619093EB0021E054
:101AD00030E0A90102C0440F551F8A95E2F74093F8
:101AE000EA001092EA008091EB0088608093EB009E
:101AF0001092E9008091E800877F86C08111A7C01D
:101B00001091C6011F778091E3008078812B80932C
:101B1000E3008091E800877F8093E8000E94470BF4
:101B20008091E80080FFFCCF8091E3008068809383
:101B3000E300111102C082E001C083E08093C30181
:101B400086C08058823008F082C08091C601909192
:101B5000C7018C3D53E0950779F583E08A838AE2DB
:101B600089834FB7F894DE01139620E03EE051E2FE
:101B7000E32FF0E050935700E49120FF03C0E2957B
:101B8000EF703F5FEF708E2F90E0EA3010F0C79655
:101B900001C0C0968D939D932F5F243149F74FBFAD
:101BA0008091E800877F8093E8006AE270E0CE01D0
:101BB00001960E94540A14C0AE014F5F5F4F6091BE
:101BC000C8010E949B09BC01892B09F440C0909177
:101BD000E800977F9093E80089819A810E94B40A77
:101BE0008091E8008B778093E80031C0803879F5E8
:101BF0008091E800877F8093E8008091BF01809307
:101C0000F1008091E8008E778093E8000E94470BF6
:101C10001EC081111CC09091C6019230C0F4809109
:101C2000E800877F8093E8009093BF010E94470BF4
:101C30008091BF01811106C08091E30087FD02C041
:101C400081E001C084E08093C3010E946608809116
:101C5000E80083FF0AC08091E800877F8093E80056
:101C60008091EB0080628093EB00AA960FB6F89407
:101C7000DEBF0FBECDBFDF91CF911F91089590932E
:101C80005901809358010895E0915801F09159014C
:101C9000309721F00190F081E02D099480E00895C3
:101CA000EF92FF920F931F93CF93DF93E091580130
:101CB000F09159013097B1F18C010280F381E02D50
:101CC00009958091AE0182FF2DC080FF04C080EE97
:101CD00092E00E949F05E80118E08AEDE82E82E07C
:101CE000F82E8091AE0180FF0BC088811F928F93E8
:101CF000FF92EF920E9438060F900F900F900F9076
:101D0000115021961111EDCF8091AE0180FF0AC0D4
:101D100088ED92E0DF91CF911F910F91FF90EF90AE
:101D20000C949F05DF91CF911F910F91FF90EF9041
:101D30000895E0915801F0915901309721F0048005
:101D4000F581E02D09940895CF93DF93EC01809104
:101D5000560190915701C817D90709F1D09357013F
:101D6000C0935601E0915801F09159013097B9F0B4
:101D70000680F781E02DCE0109958091AE0182FFAA
:101D80000EC080FF0CC0DF93CF938AEC92E09F934C
:101D90008F930E9438060F900F900F900F90DF9155
:101DA000CF910895CF93DF93EC01809154019091EE
:101DB0005501C817D90709F1D0935501C0935401B3
:101DC000E0915801F09159013097B9F00084F18504
:101DD000E02DCE0109958091AE0182FF0EC080FFFB
:101DE0000CC0DF93CF938AEB92E09F938F930E9476
:101DF00038060F900F900F900F90DF91CF910895BC
:101E00000C94C80F0E942A1B0E944A060C94521C74
:101E1000CF92DF92EF92FF920F931F93CF93DF93B6
:101E200000D000D000D0CDB7DEB70E946E068BE5A3
:101E3000C82E81E0D82E00E010E0E02E802F0E9416
:101E4000F506F60141916F01F42EF826B1F40F5F0B
:101E50001F4F0830110589F78FEF89838A831B8212
:101E60000E94331B8160782F9D838C8349815A8126
:101E70006B818D810E94FF0F47C09091AE0191FF51
:101E800004C08E830E94C90F8E8120E030E04F2D68
:101E900050E0922FBA01022E02C0759567950A9400
:101EA000E2F760FF2BC02983EA8221E030E069017C
:101EB00002C0CC0CDD1C9A95E2F790E08C219D21AC
:101EC000892B09F420E02B830E94331B8160782F3B
:101ED0009D838C8349815A816B818D810E94FF0F84
:101EE00049815A816B817C818D810E94AC1AF801F5
:101EF000E55AFE4F8081C826C08206C02F5F3F4F43
:101F00002830310531F6A3CF0E94AB1A0E94D91FA9
:101F100010915A010E94440E181741F10E94440E7C
:101F200080935A019091AE0192FF0EC090FF0CC0B9
:101F30001F928F938BEE92E09F938F930E943806AF
:101F40000F900F900F900F9080915A0126960FB628
:101F5000F894DEBF0FBECDBFDF91CF911F910F91DF
:101F6000FF90EF90DF90CF900C94BD1A26960FB69D
:101F7000F894DEBF0FBECDBFDF91CF911F910F91BF
:101F8000FF90EF90DF90CF9008950C94FB0608959A
:101F90000895EF92FF920F931F93CF93DF9384E006
:101FA00093E00E949F05C0E0D0E088E2E82E81E047
:101FB000F82E06EF12E08C2F0E94F5060E94991A67
:101FC000FF92EF921F928F93DF93CF931F930F9304
:101FD0000E94380621968DB79EB708960FB6F894E2
:101FE0009EBF0FBE8DBFC830D10529F7DF91CF91BD
:101FF0001F910F91FF90EF90089508950895CF934A
:10200000DF93CDB7DEB72B970FB6F894DEBF0FBEC8
:10201000CDBF942F4F83252F588769877A878B8769
:102020004A855B85452B21F02F3F09F59F3FF9F449
:10203000DE01119686E0FD0111928A95E9F785E0AF
:10204000FE01379601900D928A95E1F749815A81F8
:102050006B817C818D819E810E9466172B960FB6C5
:10206000F894DEBF0FBECDBFDF91CF9108954F81B1
:10207000588569857A858B850E94AC1AD9CFCF9314
:10208000882309F4A9C0C82F8238A1F40E94440E05
:1020900081FDA2C089E30E94F5190E946E1A2FEFFC
:1020A00081EE94E0215080409040E1F700C00000B4
:1020B00089E315C08338C1F40E94440E80FD8CC0B2
:1020C00083E50E94F5190E946E1A2FEF81EE94E0CD
:1020D000215080409040E1F700C0000083E50E945D
:1020E000121ACF910C946E1A8438A1F40E94440EF7
:1020F00082FD72C087E40E94F5190E946E1A2FEFCC
:1021000081EE94E0215080409040E1F700C0000053
:1021100087E4E5CF8CEF8C0F813A20F080E58C0FBF
:102120008E3248F48C2F0E943A24811155C08C2F96
:102130000E94F519D6CF80E28C0F883048F4C77022
:1021400081E001C0880FCA95EAF70E94341AC9CF0E
:102150008BE58C0F833078F4C53A29F0C63A31F01C
:1021600083E890E005C081E890E002C082E890E05A
:10217000CF910C94A40E88E58C0F853168F5C83A90
:1021800089F0C93A91F0CA3A99F0CB3AA1F0CC3A29
:10219000A9F0CD3AB1F0CE3AB9F0CF3AC1F080E033
:1021A00090E017C082EE90E014C089EE90E011C07C
:1021B0008AEE90E00EC085EB90E00BC086EB90E0DD
:1021C00008C083EB90E005C084EB90E002C087EB91
:1021D00090E0CF910C94D20ECF910895882309F40A
:1021E0006AC08238A1F40E94440E81FF64C089E372
:1021F0000E94F5190E946E1A2FEF81EE94E0215093
:1022000080409040E1F700C0000089E315C08338AA
:10221000B9F40E94440E80FF4EC083E50E94F51978
:102220000E946E1A2FEF81EE94E021508040904082
:10223000E1F700C0000083E50E94121A0C946E1AA8
:102240008438A1F40E94440E82FF35C087E40E94C6
:10225000F5190E946E1A2FEF81EE94E02150804014
:102260009040E1F700C0000087E4E6CF9CEF980FB4
:10227000913A10F390E5980F9E32F0F290E2980FA9
:10228000983050F4877091E001C0990F8A95EAF771
:10229000892F0E943A1AD2CF9BE5980F933020F4F1
:1022A00080E090E00C94A40E885A853120F480E000
:1022B00090E00C94D20E0895882321F00E94341AE5
:1022C0000C946E1A0895882321F00E943A1A0C94F7
:1022D0006E1A0895BF92CF92DF92EF92FF920F9302
:1022E0001F93CF93DF9300D000D000D0CDB7DEB7DF
:1022F00025E0FC01DE01119601900D922A95E1F78F
:10230000FC0140813181F280258122952F7063810B
:102310007481672B09F4FEC23F3F19F44F3F09F463
:10232000F9C26C0149833A8389819A812E830E9484
:10233000B419182FB92E0E94B3190E94C318EB2D9F
:10234000E295EF70F0E0E55BFF4F2E810C94F926EB
:102350008B2D807F9B2D9F70092F882311F0029574
:10236000007FFF2049F0002309F481C2802F0E94E2
:10237000471A0E946E1A7BC2812F0E94EE10002322
:1023800009F4C8C2802F0E944D1A26960FB6F89401
:10239000DEBF0FBECDBFDF91CF911F910F91FF9098
:1023A000EF90DF90CF90BF900C946E1A8B2D807FB2
:1023B0009B2D9F70092F803211F00295007F112311
:1023C00019F0113009F12AC0FF20B1F0802F22232B
:1023D00051F1213041F526960FB6F894DEBF0FBEBD
:1023E000CDBFDF91CF911F910F91FF90EF90DF90C4
:1023F000CF90BF900C94571A222319F0213009F482
:1024000089C20E945A1A2DC0FF20F1F0263008F030
:1024100081C20E94311A802329F023C0FF20F9F0E5
:10242000211116C0802F26960FB6F894DEBF0FBE7E
:10243000CDBFDF91CF911F910F91FF90EF90DF9073
:10244000CF90BF900C945C11253008F063C209C096
:10245000F601858180FF0BC28F708583E3CF211148
:102460001BC2802F82C12B2D26952695237030E02C
:102470002115310521F021303105D1F04BC2FF206B
:1024800021F0812F9B2D937002C080E090E0269672
:102490000FB6F894DEBF0FBECDBFDF91CF911F9175
:1024A0000F91FF90EF90DF90CF90BF900C94A40E0F
:1024B000FF2021F0812F9B2D937002C080E090E0DF
:1024C00026960FB6F894DEBF0FBECDBFDF91CF9139
:1024D0001F910F91FF90EF90DF90CF90BF900C94E1
:1024E000D20E812FFF2019F00E945F1E02C00E94B1
:1024F000C71E26960FB6F894DEBF0FBECDBFDF9184
:10250000CF911F910F91FF90EF90DF90CF90BF90F0
:102510000C944C1F8B2D837009F07BC0F110FAC115
:10252000812F829586958770880F880F912F9F70D5
:10253000C92ED12CE12CF12C082E04C0CC0CDD1CB2
:10254000EE1CFF1C0A94D2F714FF12C04FE050E0BB
:1025500060E070E004C0440F551F661F771F8A9526
:10256000D2F7CB01BA01609570958095909503C024
:1025700060E070E0CB012B2D269526952370422F2D
:1025800050E042305105D9F04330510569F16C29D2
:102590007D298E299F294130510551F126960FB68C
:1025A000F894DEBF0FBECDBFDF91CF911F910F9189
:1025B000FF90EF90DF90CF90BF900C94D8186C29CB
:1025C0007D298E299F2926960FB6F894DEBF0FBE6F
:1025D000CDBFDF91CF911F910F91FF90EF90DF90D2
:1025E000CF90BF900C94EA180E94D818C701B6018A
:1025F00026960FB6F894DEBF0FBECDBFDF91CF9108
:102600001F910F91FF90EF90DF90CF90BF900C94AF
:10261000C618FF2019F08B2D817001C08695882384
:1026200009F478C1812F829586958770880F880F6D
:10263000912F9F70C92ED12CE12CF12C082E04C0B3
:10264000CC0CDD1CEE1CFF1C0A94D2F714FF12C048
:102650004FE050E060E070E004C0440F551F661F7B
:10266000771F8A95D2F7CB01BA0160957095809556
:10267000909503C060E070E0CB012B2D2695269548
:102680002370422F50E042305105D9F043305105BC
:1026900069F16C297D298E299F294130510551F11D
:1026A00026960FB6F894DEBF0FBECDBFDF91CF9157
:1026B0001F910F91FF90EF90DF90CF90BF900C94FF
:1026C0008F196C297D298E299F2926960FB6F8949B
:1026D000DEBF0FBECDBFDF91CF911F910F91FF9055
:1026E000EF90DF90CF90BF900C94A1190E948F19AA
:1026F000C701B60126960FB6F894DEBF0FBECDBF58
:10270000DF91CF911F910F91FF90EF90DF90CF90CD
:10271000BF900C947D19103FC9F128F480E4810F1B
:10272000803250F09FC0123F09F461C008F44AC0E3
:10273000133F09F471C096C0012F00718B2D8F716A
:10274000FF2051F00E941619812F002319F0829565
:10275000807F69CE8F7067CE0E943719812F00234A
:1027600019F08295807F01C08F7026960FB6F8947D
:10277000DEBF0FBECDBFDF91CF911F910F91FF90B4
:10278000EF90DF90CF90BF900C946311FF20B1F0D9
:10279000253008F0BFC08B2D8F7126960FB6F894A8
:1027A000DEBF0FBECDBFDF91CF911F910F91FF9084
:1027B000EF90DF90CF90BF900C945C19263008F01A
:1027C000A9C0E9CFFF20A9F08B2D8F7126960FB6F7
:1027D000F894DEBF0FBECDBFDF91CF911F910F9157
:1027E000FF90EF90DF90CF90BF900C941619FF20D0
:1027F00059F38B2D8F7126960FB6F894DEBF0FBE5E
:10280000CDBFDF91CF911F910F91FF90EF90DF909F
:10281000CF90BF900C943719FF2099F08B2D8F71BA
:1028200026960FB6F894DEBF0FBECDBFDF91CF91D5
:102830001F910F91FF90EF90DF90CF90BF900C947D
:10284000011926960FB6F894DEBF0FBECDBFDF91FB
:10285000CF911F910F91FF90EF90DF90CF90BF909D
:102860000C94FC18FF20A9F0222309F4ADCF812F8E
:1028700026960FB6F894DEBF0FBECDBFDF91CF9185
:102880001F910F91FF90EF90DF90CF90BF900C942D
:102890003F10222309F4ADCF812F26960FB6F8946E
:1028A000DEBF0FBECDBFDF91CF911F910F91FF9083
:1028B000EF90DF90CF90BF900C94EE104B2D4F70A7
:1028C000612FC6010E94FC1B26960FB6F894DEBF4E
:1028D0000FBECDBFDF91CF911F910F91FF90EF9071
:1028E000DF90CF90BF900C940E184B2D4F70612F3E
:1028F000C60126960FB6F894DEBF0FBECDBFDF919E
:10290000CF911F910F91FF90EF90DF90CF90BF90EC
:102910000C94FF1B26960FB6F894DEBF0FBECDBFFA
:10292000DF91CF911F910F91FF90EF90DF90CF90AB
:10293000BF9008950E94541A0E94231A0E946E1A92
:102940000E9480200E944C1F80E090E00E94A40E14
:1029500080E090E00C94D20E0E94441A0C949A14D9
:102960000E94B419292F22952F7030E02C303105A8
:102970004CF42A303105C4F422503109223031059B
:1029800040F023C02C303105D1F02F303105B9F0A3
:102990001CC0853A28F48430B0F4823028F413C087
:1029A00090E2980F983078F0883E30F4803E58F4EA
:1029B0008450813A50F407C0803F39F404C093FB3F
:1029C000882780F9089581E0089580E00895CF93E5
:1029D000DF9300D000D01F92CDB7DEB70F900F90DD
:1029E0000F900F900F90DF91CF910895CF93DF93C9
:1029F00000D000D000D0CDB7DEB726960FB6F89441
:102A0000DEBF0FBECDBFDF91CF910895CF93DF938F
:102A1000C091630180916401C817A1F0D0E0CE019C
:102A200066E070E00E94C826FC01EB59FE4F408131
:102A3000518162817381848195810E94F61421966F
:102A4000C770E8CFDF91CF910895409195015091E3
:102A500096016091970170919801809199019091F0
:102A60009A010C94F614CF93DF9380919A0182958A
:102A70008F7009F05CC080919701882309F457C0DA
:102A800020916301D091640140919501C09196011C
:102A9000E0919801F09199012D1709F448C030E0B8
:102AA000309709F440C0CF3F11F44F3FE1F1C90125
:102AB00066E070E00E94C826DC01AB59BE4F11965B
:102AC0008C911197C8132FC08C9148132CC012966B
:102AD0008C911297811127C013968D919C91149718
:102AE0008E179F0708F401978E1B9F0B883C91055A
:102AF000D0F480919A018F70806180939A01C9010E
:102B000066E070E00E94C826FC01E659FE4F908105
:102B10009F709061908385E991E00E946A11DF9136
:102B2000CF910C9406152F5F3F4F2770B5CFDF91E3
:102B3000CF910895BF92CF92DF92EF92FF920F93C1
:102B40001F93CF93DF93CDB7DEB761970FB6F8949D
:102B5000DEBF0FBECDBF8C0185E0F801DE011D9602
:102B600001900D928A95E1F7D8014C9111962C9124
:102B700011971296EC9012971396CD90DC901497C3
:102B800050919501609196018091980190919901E1
:102B9000009709F46EC16F3F19F45F3F09F469C1F2
:102BA000B0909701BB2009F4C3C030919A01C816B8
:102BB000D90628F0F601E81BF90BCF0104C0809577
:102BC00090958C0D9D1DFF24F394883C910588F011
:102BD000F12C307F09F0CBC07C2DD98AC88A522FC6
:102BE0006E2D89890E94E71485E991E00E946A119F
:102BF000B4C0832F807F09F049C0621314C05413FE
:102C000012C0E11010C03F70306130939A010E94F1
:102C1000251585E991E00E946A1180919A01D801F9
:102C200015968C9331C0CD2831F12F3F11F44F3FD1
:102C300011F1FE2CE1101FC0E0916301309164019D
:102C4000E31709F45CC0F0E0CF0166E070E00E9499
:102C5000C826DC01AB59BE4F11968C9111972813F1
:102C600007C08C91481304C012968C91811103C047
:102C70003196E770E5CFFE2CEE2009F416C1809165
:102C80009A01816080939A01F12C0FC1621308C0F0
:102C9000541306C0E11004C080919A01D801C1C04C
:102CA0004D872E878D859E850E94B0148823E1F183
:102CB000EE20D1F120919A01822F82958F7090E0C1
:102CC000029774F0809195019091960198878F8377
:102CD0001986DB86CA862C87CE0107960E946A1168
:102CE00086E0F801A5E9B1E001900D928A95E1F73F
:102CF0000E9433150E942515FF24F394D6C04D87FA
:102D00002E878D859E850E94B419292F22952F70BC
:102D100030E0223031050CF0BCC09F7009F0B6C025
:102D2000805E883008F4C1C0C8010E946A11E4CFF7
:102D3000C816D90608F453C0F601E81BF90BCF01F9
:102D4000883C910508F450C0F12C7C2DD98AC88AA2
:102D5000522F6E2D89890E94E714E5E9F1E086E0A3
:102D6000DF011D928A95E9F70E9425159EC0621326
:102D700014C0541312C0E11010C080919A01F801E0
:102D80008583C8010E946A1186E0E5E9F1E0DF0170
:102D90001D928A95E9F7FB2C88C04D872E878D857B
:102DA0009E850E94B014882309F4BECFEE2009F45A
:102DB000BBCF20919A01822F82958F7090E002976D
:102DC0000CF48ECF80919501909196019A8389831E
:102DD0001B82DD82CC822E83CE0101967FCF80952F
:102DE00090958C0D9D1DACCFFE2CEE2009F49CCF50
:102DF00062132EC054132CC020919A0120FD1FC0D5
:102E0000822F82958F70D9F0D80115962C93159743
:102E10008F3049F08F5F982F9295907F822F8F701F
:102E2000892B15968C93C8010E946A1186E0F801DF
:102E3000A5E9B1E001900D928A95E1F795CF86E082
:102E4000F801A5E9B1E001900D928A95E1F72DC056
:102E50004D872E878D859E850E94B014811140CFAD
:102E600080919A01816080939A01C8010E946A1141
:102E70001CC0EE2009F458CF4D872E878D859E8586
:102E80000E94B014882309F44FCF2ACF811148CF74
:102E90000CC0243031050CF047CF9F7009F440CFAF
:102EA000F8019581907F09F03BCF8F2D61960FB689
:102EB000F894DEBF0FBECDBFDF91CF911F910F9170
:102EC000FF90EF90DF90CF90BF900895CF93DF9366
:102ED000CDB7DEB72C970FB6F894DEBF0FBECDBFCF
:102EE0004F83588769877A878B879C87CE0107969F
:102EF0000E949A15882371F08F8198852A853B85D9
:102F0000232B09F43FC09F3F09F068C08F3F09F0B1
:102F100065C038C086E0FE013796DE01119601904B
:102F20000D928A95E1F76F817885EA85FB85309768
:102F300049F17F3F11F46F3F29F18091640190E0E6
:102F40009C012F5F3F4F277033274091630150E072
:102F50002417350709F44BC069837A83FD83EC831A
:102F600066E070E00E94C826DC01AB59BE4F96E0D7
:102F7000FE01319601900D929A95E1F7209364013C
:102F80000E94061580916301909164018917E9F10F
:102F900090E066E070E00E94C8268B599E4F0E9428
:102FA0009A15882391F18091630190E066E070E0CA
:102FB0000E94C826FC01EB59FE4F4081518162817D
:102FC0007381848195810E94F6148091630190E061
:102FD00001968770992780936301D4CF4F815885DC
:102FE00069857A858B859C850E94F614CBCF0E94DB
:102FF000AC141092640110926301E5E9F1E086E0FF
:10300000DF011D928A95E9F7BDCF2C960FB6F89493
:10301000DEBF0FBECDBFDF91CF910895DF92EF925B
:10302000FF920F931F93CF93DF93FC01892B09F439
:103030008AC0E12CF12CDD24D394EF0121968491F8
:10304000853709F461C058F4843708F04EC08430E5
:1030500008F06AC08130D1F0823071F174C08837D5
:1030600009F45DC050F4863709F455C0873709F07C
:103070006AC08E2D0E94411A54C09CE7980F903769
:1030800008F061C08F770E94EE1050C08F010E5F74
:103090001F4FFE01849190E2980F983050F4877092
:1030A000FD2D01C0FF0F8A95EAF78F2F0E94471A66
:1030B00014C00E943F1013C08F010E5F1F4FFE010E
:1030C000C49180E28C0F883060F4C7708D2D01C0F0
:1030D000880FCA95EAF70E944D1A0E946E1AE801FD
:1030E00025C08C2F0E94EE10FACF9F012E5F3F4F1C
:1030F000FE01C491CC2369F08FE99FE00197F1F7BD
:1031000000C00000C150F6CF9F012E5F3F4FFE016F
:10311000F490E9010BC00E94311AE82E07C00E940A
:10312000441A0E946E1A02C00E943F108F2D8823FD
:1031300041F0EFE9FFE03197F1F700C00000815066
:10314000F6CFFE017ACFDF91CF911F910F91FF90C3
:10315000EF90DF90089560939F017093A00180939A
:10316000A1019093A2010E94BB1A0C949A1460933F
:103170009B0170939C0180939D0190939E010E94FE
:10318000BC1A0C949A1408950C94AB180F931F93C7
:1031900000919F011091A0012091A1013091A20105
:1031A000602B712B822B932B1F910F910C94AB18DA
:1031B0000F931F9300919F011091A0012091A101F5
:1031C0003091A20160237123822393231F910F91D9
:1031D0000C94AB180F931F9300919F011091A001C5
:1031E0002091A1013091A2016027712782279327A6
:1031F0001F910F910C94AB1860E070E0CB010C9420
:10320000B7180F931F9341E050E060E070E08A012F
:103210009B0104C0000F111F221F331F8A95D2F794
:10322000C901B8011F910F910C94B7180F931F9308
:1032300041E050E060E070E004C0440F551F661F9D
:10324000771F8A95D2F780919B0190919C01A09164
:103250009D01B0919E018A019B01082B192B2A2BFD
:103260003B2BC901B8011F910F910C94B7180F9314
:103270001F9341E050E060E070E004C0440F551F30
:10328000661F771F8A95D2F7409550956095709587
:1032900080919B0190919C01A0919D01B0919E0114
:1032A0008A019B01082319232A233B23C901B80162
:1032B0001F910F910C94B7180F931F9341E050E0AA
:1032C00060E070E004C0440F551F661F771F8A95A9
:1032D000D2F780919B0190919C01A0919D01B091AA
:1032E0009E018A019B01082719272A273B27C9012C
:1032F000B8011F910F910C94B7180F931F93009171
:103300009B0110919C0120919D0130919E01602BA9
:10331000712B822B932B1F910F910C94B7180F9345
:103320001F9300919B0110919C0120919D01309170
:103330009E0160237123822393231F910F910C948C
:10334000B7180F931F9300919B0110919C0120913E
:103350009D0130919E0160277127822793271F913D
:103360000F910C94B7180895CF92DF92EF92FF92CD
:103370000F931F93CF93DF938C01C0909F01D09048
:10338000A001E090A101F090A20140919B01509119
:103390009C0160919D0170919E01C42AD52AE62A64
:1033A000F72ACFE1D0E0D701C6010C2E04C0B695B4
:1033B000A795979587950A94D2F780FF07C0B80123
:1033C0008C2F0E94CD1B8130910531F4219758F745
:1033D000B80180E00E94CD1BDF91CF911F910F912A
:1033E000FF90EF90DF90CF90089520910C013091E5
:1033F0000D01F90132969FEF40E05191581789F085
:103400009F3F19F4511101C0942F4F5F4630A9F727
:103410009F3F39F0F901E90FF11D97FDFA9582837D
:103420000895089520910C0130910D01F901329613
:10343000285F3F4F9081981301C010823196E217A8
:10344000F307C1F7089581E090E0E0910C01F0915D
:103450000D01E80FF91F1082019688309105A9F738
:1034600008958091AD0108959091AD01892B8093CD
:10347000AD01089580959091AD0189238093AD01B0
:1034800008958093AD0108951092AD010895909133
:10349000AC01892B8093AC01089580959091AC018B
:1034A00089238093AC0108951092AC010895809314
:1034B000A30108951092A301089580910C019091A9
:1034C0000D01FC0131969C01285F3F4F80E09191F6
:1034D00091118F5FE217F307D1F70895E0910C0186
:1034E000F0910D018091AD018083E0910C01F0918C
:1034F0000D0190818091AC01892B80838091A30183
:10350000882361F0E0910C01F0910D019081892BED
:1035100080830E945D1A81111092A30180910C0199
:1035200090910D010C94500E9093350180933401CD
:1035300008958295982F9C7C292F26952695982F63
:103540009373990F990F922B892F8A7A8695957587
:10355000990F892B08950895CF93DF9300D000D061
:103560001F92CDB7DEB70F900F900F900F900F9076
:10357000DF91CF910895089508950C94C50F089593
:103580008091C301843021F11092AF0120E488E1E1
:1035900090E00FB6F894A895809360000FBE20933A
:1035A000600083B7817F846083BF83B7816083BFFE
:1035B0007894889583B78E7F83BF0FB6F894A895CB
:1035C00080916000886180936000109260000FBE5F
:1035D0000895CF930E94FD0F0E946E060E94FE0F79
:1035E000C0E08C2F0E94F506811104C0CF5FC83067
:1035F000C1F701C081E0CF9108950E94C70F0C94DC
:10360000AC141F920F920FB60F9211248F939F93B9
:10361000AF93BF938091AF01811113C08091B0012E
:103620009091B101A091B201B091B3014196A11D59
:10363000B11D8093B0019093B101A093B201B093FA
:10364000B301BF91AF919F918F910F900FBE0F90DB
:103650001F90189582E084BD93E095BD9AEF97BDC9
:1036600080936E0008952FB7F8948091B0019091E7
:10367000B101A091B201B091B3012FBF08952FB74E
:10368000F8946091B0017091B1018091B201909174
:10369000B3012FBF0895CF92DF92EF92FF920F9365
:1036A0001F932FB7F8944091B0015091B1016091F0
:1036B000B2017091B3012FBF6A017B01EE24FF2498
:1036C0008C0120E030E0C016D106E206F30610F4CB
:1036D000415051099A01281B390BC9011F910F91C3
:1036E000FF90EF90DF90CF9008951F920F920FB64A
:1036F0000F9211248F939F93AF93BF938091B0014A
:103700009091B101A091B201B091B3010196A11DB8
:10371000B11D8093B0019093B101A093B201B09319
:10372000B301BF91AF919F918F910F900FBE0F90FA
:103730001F9018950E94980BF8942FEF87EA91E656
:10374000215080409040E1F700C0000087E090EBFE
:10375000DC018093CD019093CE01A093CF01B09373
:10376000D0019CE088E10FB6F894A89580936000A2
:103770000FBE90936000FFCFE92FF0E093E0EE0FD3
:10378000FF1F9A95E1F7E80FF11DEA54FF4F94915E
:10379000892F8F7092959F700895CF93C82FCB017A
:1037A0000E94BC1B492F90E0242F30E054E0220FF0
:1037B000331F5A95E1F7282B392B2038310519F49E
:1037C00080E090E017C0EC2FF0E023E0EE0FFF1F49
:1037D0002A95E1F74770E40FF11D34E0EE0FFF1F6B
:1037E0003A95E1F7E80FF91FEE0FFF1FE050F84997
:1037F00085919491CF91089580E090E00895089587
:10380000CF92DF92EF92FF920F931F93CF936C01B1
:10381000C0E08C2F0E94F50600E010E0E82EF12CAD
:10382000C701002E02C0959587950A94E2F780FFA4
:1038300016C0602F7C2F80E00E94CD1B9C018C1550
:103840009D0559F0832F807E932F907C11F0803A54
:1038500031F430E02C153D0511F481E009C00F5F13
:103860001F4F08301105E1F6CF5FC83091F680E0B8
:10387000CF911F910F91FF90EF90DF90CF9008951F
:10388000CF93DF93EC018CE290E00E94001C882330
:1038900029F0CE01DF91CF910C94001C80E0DF91E4
:1038A000CF910895CF930E94B31D811102C00E9451
:1038B000991D89E193E00E949F05C5E6C15049F03A
:1038C0000E946E068FE39CE90197F1F700C00000AB
:1038D000F5CF82E193E00E949F0589E290E00E948B
:1038E000401C811124C18AE290E00E94401C811199
:1038F0000E94991D85E090E00E94401C81110E9469
:103900009A1B0E94BF1A0E94BE1D8093AE0187E0E1
:1039100090E00E94401C8823C1F18BE190E00E945E
:10392000401C882351F08091AE0181FB222720F9B1
:1039300091E0922790FB81F90FC08EE090E00E9409
:10394000401C882361F08091AE0182FB222720F980
:1039500091E0922790FB82F98093AE0116C080E13E
:1039600090E00E94401C9091AE01882341F093FBAF
:10397000222720F981E0822780FB93F904C0892F58
:10398000809580FB90F99093AE018091AE010E94EA
:10399000C21D0E94D01D8093CC0180EE90E00E9459
:1039A000401C882341F08091CC01982F909590FB8A
:1039B00080F98093CC0189E390E00E94401C882329
:1039C00059F08091CC0181FB222720F991E09227C8
:1039D00090FB81F98093CC0182EE90E00E94401C24
:1039E000882359F08091CC0182FB222720F991E0B5
:1039F000922790FB82F98093CC0186EE90E00E94A2
:103A0000401C882359F08091CC0183FB222720F9A8
:103A100091E0922790FB83F98093CC0183EE90E0B4
:103A20000E94401C882359F08091CC0184FB2227FE
:103A300020F991E0922790FB84F98093CC0185E3F3
:103A400090E00E94401C882359F08091CC0185FBB6
:103A5000222720F991E0922790FB85F98093CC01F1
:103A600081E390E00E94401C882359F08091CC01B2
:103A700086FB222720F991E0922790FB86F980931C
:103A8000CC0181E190E00E94401C882359F0809194
:103A9000CC0187FB222720F991E0922790FB87F940
:103AA0008093CC018091CC010E94D41D87E290E0EC
:103AB0000E94401CC82F8EE190E00E94401C8111A2
:103AC000C2608FE190E00E94401C8111C46080E2DE
:103AD00090E00E94401C8111C86081E290E00E9449
:103AE000401C8111C06182E290E00E94401C811163
:103AF000C06283E290E00E94401C8111C06484E2B5
:103B000090E00E94401C882311F0C06802C0CC23C2
:103B100029F08C2F0E94CB1D6C2F03C00E94C71D63
:103B2000682F70E080E090E0CF910C94C418CF91A2
:103B300008956DEE7EEF80E090E00E942F2760E018
:103B400082E090E00E94212760E083E090E00E9404
:103B5000212760E084E090E00E94212760E085E07A
:103B600090E00C94212780E090E00E941B2721E048
:103B70008D3E9E4F09F020E0822F089582E090E074
:103B80000C941327682F82E090E00C94212783E0A7
:103B900090E00C941327682F83E090E00C94212789
:103BA00084E090E00C941327682F84E090E00C945C
:103BB00021278091B60180FF0CC08091110190E017
:103BC00065E070E00E94C826959587959595879544
:103BD0002EC081FF0AC08091110190E065E070E085
:103BE0000E94C8269595879522C082FF08C08091C3
:103BF000110190E065E070E00E94C82618C0209195
:103C0000B7012223D1F030911001231780F7809162
:103C1000110190E065E070E00E94C826622F70E01C
:103C20000E94C826632F70E00E94E526CB018038F1
:103C3000910530F4009731F0089585E090E0089503
:103C40008FE7089581E008958091B60180FF08C054
:103C500060910F0170E0759567957595679523C024
:103C600081FF06C060910F0170E0759567951BC0DC
:103C700082FF04C060910F0170E012C06091B70133
:103C80006623D1F020910E016217A0F780910F01F9
:103C900070E090E00E94C826622F70E00E94E52646
:103CA0006038710528F46115710521F0862F08959B
:103CB0008FE7089581E0089561E070E0F4CF803FE0
:103CC00021F40E94D91D819504C0813F29F40E94EE
:103CD000D91D8093BA010895823F21F40E94D91D15
:103CE000819504C0833F29F40E94D91D8093B901B6
:103CF0000895893F19F40E94241E05C08A3F31F4BB
:103D00000E94241E81958093BB0108958B3F21F46E
:103D10000E94241E819504C08C3F29F40E94241E19
:103D20008093BC010895843F21F48091B8018160A3
:103D300017C0853F21F48091B801826011C0863F91
:103D400021F48091B80184600BC0873F21F48091F9
:103D5000B801886005C0883F31F48091B801806166
:103D60008093B80108958D3F21F48091B601816060
:103D70000BC08E3F21F48091B601826005C08F3F59
:103D800029F48091B60184608093B6010895803F44
:103D900039F48091BA0187FF6CC01092BA0169C0F2
:103DA000813F29F48091BA011816BCF362C090914A
:103DB000B901823F29F497FF5CC01092B90159C044
:103DC000833F19F41916CCF354C0893F41F4809114
:103DD000BB0118160CF04DC01092BB014AC08A3FBF
:103DE00029F48091BB0187FF44C0F6CF8B3F39F4A3
:103DF0008091BC0187FF3DC01092BC013AC08C3F4E
:103E000029F48091BC011816BCF333C0843F21F41F
:103E10008091B8018E7F17C0853F21F48091B80151
:103E20008D7F11C0863F21F48091B8018B7F0BC03C
:103E3000873F21F48091B801877F05C0883F31F426
:103E40008091B8018F7E8093B80113C08D3F21F41B
:103E50008091B6018E7F0BC08E3F21F48091B60118
:103E60008D7F05C08F3F29F48091B6018B7F8093B1
:103E7000B6018091B90181110EC08091BA01811102
:103E80000AC08091BB01811106C08091BC018111E3
:103E900002C01092B70108958091AE0183FF7EC0E9
:103EA00085E593E00E949F058091B8011F928F9352
:103EB00080E593E09F938F930E9438068EE493E011
:103EC0000E949F058091B901282F082E000C330B0A
:103ED0003F938F938BE493E09F938F930E943806D8
:103EE00089E493E00E949F058091BA01282F082E53
:103EF000000C330B3F938F9386E493E09F938F9353
:103F00000E94380684E493E00E949F058091BB01E3
:103F1000282F082E000C330B3F938F9381E493E0FE
:103F20009F938F930E9438068FE393E00E949F0532
:103F30008091BC01282F082E000C330B3F938F93E8
:103F40008CE393E09F938F930E94380689E393E07C
:103F50000E949F058091B7011F928F9386E393E0A3
:103F60009F938F930E94380684E393E00E949F05FD
:103F70008091B6011F928F9381E393E09F938F937B
:103F80000E9438068EE293E00E949F058DB79EB78F
:103F90004C960FB6F8949EBF0FBE8DBF88EB91E094
:103FA0000E94990E0E94331B9093B5018093B40137
:103FB00008951F93CF93DF938091B4019091B50141
:103FC0000E944B1BFC012091B701222329F0909104
:103FD0001201892F90E007C08091130190E06AE000
:103FE00070E00E94C826E817F90708F485C08091A0
:103FF000B901C091BA01D091BB011091BC018111EE
:1040000007C0C11175C0D11173C0111171C074C046
:104010002F3F19F02F5F2093B701181624F40E9448
:10402000D91D8093B9018091B90187FF05C00E9415
:10403000D91D81958093B9011C1624F40E94D91DC5
:104040008093BA018091BA0187FF05C00E94D91DF3
:1040500081958093BA016091B901662331F1C091D5
:10406000BA01CC2311F1062E000C770B880B990BAB
:104070000E94C72523E333E343E35FE30E942B263B
:104080000E948F256093B9016C2FCC0F770B880BA2
:10409000990B0E94C72523E333E343E35FE30E94C8
:1040A0002B260E948F256093BA011D1624F40E94CE
:1040B000241E8093BB018091BB0187FF05C00E9435
:1040C000241E81958093BB01111624F40E94241EA6
:1040D0008093BC018091BC0187FF05C00E94241E13
:1040E00081958093BC01DF91CF911F910C944C1F5F
:1040F0002F3F09F08FCF97CFDF91CF911F91089578
:10410000E8EBF1E085E0DF011D928A95E9F7109276
:10411000B7011092B601089588E795E00E949F05C7
:104120001F9281E08F931F9285E08F938AE295E042
:104130009F938F930E9438060F900F900F900F90CF
:104140000F900F9008958330E9F128F4813061F0E9
:10415000823009F10895853009F462C008F449C03D
:10416000863009F474C0089580911301262F30E041
:10417000280F311D2F3F310524F4680F6093130180
:1041800003C08FEF80931301809113011F928F93CF
:1041900083E694E072C080911201262F30E0280F50
:1041A000311D2F3F310524F4680F6093120103C0C5
:1041B0008FEF80931201809112011F928F9381E5FE
:1041C00094E05BC080911101262F30E0280F311D53
:1041D0002F3F310524F4680F6093110103C08FEF66
:1041E00080931101809111011F928F938EE394E0CF
:1041F00044C080911001262F30E0280F311D2F3F41
:10420000310524F4680F6093100103C08FEF809391
:104210001001809110011F928F9389E294E02DC0CC
:1042200080910F01262F30E0280F311D2F3F3105DF
:1042300024F4680F60930F0103C08FEF80930F0188
:1042400080910F011F928F9380E194E016C08091BE
:104250000E01262F30E0280F311D2F3F310524F4A9
:10426000680F60930E0103C08FEF80930E01809161
:104270000E011F928F9385EF93E09F938F930E947F
:1042800038060F900F900F900F900895833081F1B2
:1042900028F4813059F08230D1F00895853009F446
:1042A00049C0B8F1863009F456C0089580911301D1
:1042B000681720F4861B8093130102C0109213012B
:1042C000809113011F928F9386EE93E054C08091EA
:1042D0001201681720F4861B8093120102C010920D
:1042E0001201809112011F928F9384ED93E043C0DD
:1042F00080911101681720F4861B8093110102C080
:1043000010921101809111011F928F9381EC93E023
:1043100032C080911001681720F4861B8093100131
:1043200002C010921001809110011F928F938CEAAD
:1043300093E021C080910F01681720F4861B8093C1
:104340000F0102C010920F0180910F011F928F93F5
:1043500083E993E010C080910E01681720F4861B5A
:1043600080930E0102C010920E0180910E011F92E7
:104370008F9388E793E09F938F930E9438060F9066
:104380000F900F900F900895CF93C82F1F928F9387
:104390008DE796E09F938F930E94380681E090E02E
:1043A000A0E0B0E0BC01CD0104C0660F771F881FFC
:1043B000991FCA95D2F70E94C4180F900F900F90C2
:1043C0000F90CF910C94AC14CF938732B0F58E310F
:1043D00008F040C28E3009F4BEC100F5873009F400
:1043E0008DC1A8F4863009F039C28091AE01817F79
:1043F0008E7F8093AE0182E896E00E949F0585E85B
:104400009AE00E949F0581E08093BE0175C18830CB
:1044100009F43FC08B3009F46BC120C2863109F426
:10442000E0C120F4803109F4AAC118C2893109F42D
:10443000C1C18B3109F47BC111C2883309F458C161
:1044400050F4893209F404C2853309F401C2873279
:1044500009F004C2FDC1833409F4FAC128F48A3397
:1044600008F4FCC18953F7C1883409F0F7C10E94F0
:10447000AC1484E79AE00E949F059FEF23ED80E350
:10448000915020408040E1F700C000000E949A1B3C
:1044900033C189E89AE00E949F0589E798E00E946D
:1044A0009F050E94C71D1F928F9386E798E09F93F8
:1044B0008F930E94380684E798E00E949F050E942F
:1044C000BE1DC82F81E698E00E949F051F92CF93E2
:1044D0008CE598E09F938F930E9438068AE598E0D8
:1044E0000E949F0580E598E00E949F058C2F8170B7
:1044F0001F928F938DE498E09F938F930E943806CC
:104500008BE498E00E949F0581E498E00E949F055B
:10451000C1FB882780F91F928F938EE398E09F93C9
:104520008F930E9438068CE398E00E949F0580E3F9
:1045300098E00E949F05C2FB882780F91F928F9305
:104540008DE298E09F938F930E9438068BE298E06B
:104550000E949F0582E298E00E949F05C3FBCC2742
:10456000C0F91F92CF938FE198E09F938F930E94A1
:1045700038068DE198E00E949F050E94D01DC82F4B
:1045800089E098E00E949F051F92CF9384E098E015
:104590009F938F930E94380682E098E00E949F05C7
:1045A00089EE97E00E949F058C2F81701F928F9358
:1045B00086EE97E09F938F930E9438068DB79EB743
:1045C00080960FB6F8949EBF0FBE8DBF84EE97E025
:1045D0000E949F058DEC97E00E949F05C1FB8827F4
:1045E00080F91F928F938AEC97E09F938F930E949C
:1045F000380688EC97E00E949F0586EB97E00E94C2
:104600009F05C2FB882780F91F928F9383EB97E069
:104610009F938F930E94380681EB97E00E949F053D
:104620008FE997E00E949F05C3FB882780F91F92BE
:104630008F938CE997E09F938F930E9438068AE9C5
:1046400097E00E949F0580E997E00E949F05C4FBC8
:10465000882780F91F928F938DE897E09F938F931F
:104660000E9438068BE897E00E949F0589E797E053
:104670000E949F05C5FB882780F91F928F9386E7CC
:1046800097E09F938F930E94380684E797E00E94FB
:104690009F0588E597E00E949F05C6FB882780F963
:1046A0001F928F9385E597E09F938F930E94380622
:1046B00083E597E00E949F058BE497E00E949F05A9
:1046C000C7FBCC27C0F91F92CF9388E497E09F9354
:1046D0008F930E94380686E497E00E949F058DB76D
:1046E0009EB74C960FB6F8949EBF0FBE8DBF04C008
:1046F00089EA96E00E949F05C1E0B5C08091AE01B5
:10470000C82FC17080FF09C087E69AE00E949F050C
:104710008091AE01817F8E7F47C08BE59AE00E9439
:104720009F058091AE0181608093AE01E5CF9091AD
:10473000AE0191FBCC27C0F981E0C827892FC0FBCF
:1047400081F98093AE01CC2319F08EE49AE027C062
:1047500080E49AE0CFCF9091AE0192FBCC27C0F9D4
:1047600081E0C827892FC0FB82F98093AE01CC235A
:1047700019F081E39AE013C081E29AE0BBCF9091F7
:10478000AE0193FBCC27C0F981E0C827892FC0FB7D
:1047900083F98093AE01CC2351F085E19AE00E9429
:1047A0009F058091AE0181608093AE015CC088E07E
:1047B0009AE0A0CF89EF99E00E949F0581ED99E0F2
:1047C0000E949F058FE999E00E949F0582E799E08A
:1047D0000E949F0583E299E00E949F0584EF98E084
:1047E00089CF86EE98E00E949F050E94440E1F929A
:1047F0008F938CEC98E09F938F930E943806809162
:104800000B011F928F9385EB98E09F938F930E94EB
:104810003806809153011F928F9382EA98E09F930C
:104820008F930E9438060E943F1B9F938F937F9324
:104830006F938BE898E09F938F930E9438068DB713
:104840009EB742960FB6F8949EBF0FBE8DBF54CF51
:1048500080E001C08D510E94C4214ECF89E898E0CC
:104860000E949F05C0E08C2FCF91089580E00895AD
:1048700080E00895CF93C82F8091BE01813071F000
:1048800020F0823009F44BC042C1E0910C01F0915C
:104890000D018081823209F03CC107C0E0910C011A
:1048A000F0910D018081823261F48C2F0E943624B8
:1048B000811104C08C2F0E94E4212FC081E090E080
:1048C0002CC08C2F0E943824811126C0C431E1F005
:1048D00070F4CB3081F0C031D1F40E948C2085E798
:1048E00096E00E949F0582E08093BE0115C0C93208
:1048F00059F0C83361F482E896E00E949F0589E789
:1049000096E00E949F0508C01092BE0104C183E793
:1049100096E00E949F05FFC081E08170FEC0C43216
:1049200028F5CE3108F0C1C0CB30A1F1D0F4C730AA
:1049300009F0D3C08EE18093130182E380931201CA
:104940008AE08093110184E18093100188E08093D4
:104950000F0188E280930E0189E195E00E949F0596
:10496000BFC0C33149F1C431C1F0B7C0CB3409F481
:10497000A9C028F4C93289F0C83361F0AEC0C1358E
:1049800009F49EC0C23509F499C0CE3409F0A5C01F
:104990006AE09EC00E948C20A3C08091BD01882344
:1049A00019F01092BD019CC086E295E00E949F051F
:1049B00081E08093BE01B1C080E095E00E949F0538
:1049C0008EEE94E00E949F05809113011F928F93B9
:1049D0008BEE94E09F938F930E94380689EE94E0CB
:1049E0000E949F0587ED94E00E949F05809112012F
:1049F0001F928F9384ED94E09F938F930E943806CB
:104A000082ED94E00E949F0583EC94E00E949F0554
:104A1000809111011F928F9380EC94E09F938F936C
:104A20000E9438068EEB94E00E949F058DEA94E088
:104A30000E949F05809110011F928F938AEA94E053
:104A40009F938F930E94380688EA94E00E949F0506
:104A500083E994E00E949F0580910F011F928F933C
:104A600080E994E09F938F930E9438068EE894E04B
:104A70000E949F0587E794E00E949F0580910E01A8
:104A80001F928F9384E794E09F938F930E94380640
:104A900082E794E00E949F058DB79EB748960FB6B7
:104AA000F8949EBF0FBE8DBF1BC0CE51EC2FF0E01F
:104AB000E75DFE4F80818093BD0112C061E003C0BD
:104AC00061E006C06AE08091BD010E94A32008C099
:104AD0008091BD010E94462103C087E195E013C08B
:104AE0008091BD01882369F01F928F9381E195E049
:104AF0009F938F930E9438060F900F900F900F9006
:104B000004C08EE095E00E949F0581E006C01092EF
:104B1000BE0180E002C080E000CFCF9108950E94E6
:104B200096256894B1110C94252608950E940A26B2
:104B300088F09F5798F0B92F9927B751B0F0E1F05E
:104B4000660F771F881F991F1AF0BA95C9F714C00E
:104B5000B13091F00E942426B1E008950C942426EF
:104B6000672F782F8827B85F39F0B93FCCF3869547
:104B700077956795B395D9F73EF4909580957095A4
:104B800061957F4F8F4F9F4F0895E89409C097FB21
:104B90003EF490958095709561957F4F8F4F9F4F14
:104BA0009923A9F0F92F96E9BB279395F695879558
:104BB00077956795B795F111F8CFFAF4BB0F11F41B
:104BC00060FF1BC06F5F7F4F8F4F9F4F16C08823C2
:104BD00011F096E911C0772321F09EE8872F762FF8
:104BE00005C0662371F096E8862F70E060E02AF039
:104BF0009A95660F771F881FDAF7880F9695879525
:104C000097F9089557FD9058440F551F59F05F3F8D
:104C100071F04795880F97FB991F61F09F3F79F0DE
:104C200087950895121613061406551FF2CF469560
:104C3000F1DF08C0161617061806991FF1CF8695E2
:104C40007105610508940895E894BB2766277727C6
:104C5000CB0197F908950E943D260C94B7260E9437
:104C6000A92638F00E94B02620F0952311F00C946C
:104C7000A0260C94A6260C9425260E94022678F3E2
:104C80009923C9F35523B9F3950F50E0551FAA276F
:104C9000EE27FF27BB2700240894679520F4E20F36
:104CA000F31FB41F0A1E220F331F441FAA1F66954D
:104CB000A9F7779530F4F30FB41F0A1E121E08F4FB
:104CC0006395330F441FAA1F221F769599F7879586
:104CD00020F4B40F0A1E121E631F440FAA1F221FC6
:104CE000331F8695A9F7862F712D602D11249F57AC
:104CF00050409AF0F1F088234AF0EE0FFF1FBB1FDF
:104D0000661F771F881F91505040A9F79E3F51059D
:104D100080F00C94A0260C9425265F3FE4F3983E87
:104D2000D4F3869577956795B795F795E7959F5F47
:104D3000C1F7FE2B880F911D9695879597F90895D9
:104D400097F99F6780E870E060E008959FEF80EC3E
:104D5000089500240A9416161706180609060895E1
:104D600000240A9412161306140605060895092E47
:104D70000394000C11F4882352F0BB0F40F4BF2BB6
:104D800011F460FF04C06F5F7F4F8F4F9F4F0895F6
:104D90000024552704C0080E591F880F991F00973B
:104DA00029F076956795B8F37105B9F7802D952FA1
:104DB0000895991B79E004C0991F961708F0961B77
:104DC000881F7A95C9F78095089597FB072E16F4EA
:104DD000009407D077FD09D00E94FF2607FC05D07C
:104DE0003EF4909581959F4F0895709561957F4F02
:104DF0000895EE0FFF1F0590F491E02D0994AA1B72
:104E0000BB1B51E107C0AA1FBB1FA617B70710F0B5
:104E1000A61BB70B881F991F5A95A9F780959095E7
:104E2000BC01CD010895F999FECF92BD81BDF89ADC
:104E3000992780B50895A8E1B0E042E050E00C94D5
:104E40003627262FF999FECF1FBA92BD81BD20BD0E
:104E50000FB6F894FA9AF99A0FBE019608950E9437
:104E60002127272F0C942227DC01CB01FC01F99983
:104E7000FECF06C0F2BDE1BDF89A319600B40D92A6
:0C4E800041505040B8F70895F894FFCF5F
:104E8C00050307F407D1079D07690701A40128084A
:104E9C00140A321E404D36227A022D02F701D5013A
:104EAC0061017A019301AC010001020304050607BC
:044EBC0008090000E1
:106800000000000000000000040005000600070072
:10681000080009000A000B000C000D000E000F001C
:1068200010001100120013001400150016001700CC
:10683000180019001A001B001C001D001E001F007C
:10684000200021002200230024002500260027002C
:10685000280029002A002B002C002D002E002F00DC
:1068600030003100000033003400350036003700BE
:106870003800E00000000000000000000000000000
:106880000000000000000000000000000000000008
:1068900000000000000000000000000000000000F8
:1068A00000000000000000000000000000000000E8
:1068B00000000000000000000000000000000000D8
:1068C00000000000000000006400650000000000FF
:1068D00000000000000000000000000000000000B8
:1068E0000000000000000000320000000000000076
:1068F000E000E100E200E300E400E500E600E7A1DB
:106900000000000000000000EA4401000100E24431
:106910000100010001005500460054004A004B00F0
:10692000560057004700480001000100E9440100FB
:106930000100010001000100010001003A003B00DC
:106940003C003D003E003F0040004100420043004B
:10695000580001004C00390001004400450052007D
:1069600001002A00000050004F0029004D004E0099
:1069700051000100000000000000000000000000C5
:106980000000000000000000000000000000000007
:1069900000000000000000000000000000000000F7
:1069A00000000000000000000000000000000000E7
:1069B00000000000000000000000000000000000D7
:1069C00000000000000000000100010000000000C5
:1069D00000000000000000000000000000000000B7
:1069E000000000000000000049000000000000005E
:1069F000010001000100010001000100010001008F
:00000001FF
